:100000000AC021C020C01FC01EC01DC08DC11BC0A2
:100010001AC019C018C011241FBE20E0A89521BD28
:1000200020E025BFE8ECF7E0A0E6B0E003C0C8950B
:1000300031960D92A437D9F7A4E7B0E001C01D9224
:10004000A039E9F73DC300C01895CF93DF93CDB732
:10005000DEB72E970FB6F894DEBF0FBECDBF8091EE
:1000600088009091890068E572E098D3972F862FD9
:1000700080937600809188009091890068E572E015
:100080008DD389839A8389819A816CE370E086D3CA
:10009000972F862F8093770089819A816CE370E097
:1000A0007DD389839A8389819A816AE070E076D3CF
:1000B000972F862F8093780089819A816AE070E07B
:1000C0006DD389839A838981809379002E960FB6A8
:1000D000F894DEBF0FBECDBFDF91CF910895CF93CF
:1000E000DF93CDB7DEB780917600992768E572E09F
:1000F00044D3282F392F8091770099276CE370E043
:100100003CD3532F422F480F591F80917800282F3E
:100110003327932F822F880F991F880F991F880FDD
:10012000991F820F931F820F931F242F352F280FA3
:10013000391F809179009927820F931F909389002E
:1001400080938800DF91CF910895CF93DF93CDB74F
:10015000DEB721970FB6F894DEBF0FBECDBF00000B
:100160008827E19B8395898389818823C9F3219618
:100170000FB6F894DEBF0FBECDBFDF91CF910895CB
:10018000CF93DF93CDB7DEB7E0DF80E190E0C3D25D
:1001900080937600DADF80E290E0BDD28093770032
:1001A000D4DF80E390E0B7D280937800CEDF80E4A4
:1001B00090E0B1D28093790092DFDF91CF910895E2
:1001C000CF93DF93CDB7DEB7C0DF80E190E0A3D25D
:1001D000982F80917600891731F0B7DF6091760013
:1001E00080E190E0ADD2B1DF80E290E094D2982F30
:1001F00080917700891731F0A8DF6091770080E265
:1002000090E09ED2A2DF80E390E085D2982F80918B
:100210007800891731F099DF6091780080E390E0F1
:100220008FD293DF80E490E076D2982F809179008E
:10023000891731F08ADF6091790080E490E080D204
:10024000DF91CF910895CF93DF93CDB7DEB71092B2
:1002500083001092820080918200909183008F3FF2
:10026000910508F00BC000008091820090918300FE
:1002700001969093830080938200EDCFDF91CF9120
:100280000895CF93DF93CDB7DEB71092750010922B
:10029000740080917400909175002BE0883B920768
:1002A00008F00BC0D0DF809174009091750001962A
:1002B0009093750080937400ECCFDF91CF910895F7
:1002C000CF93DF93CDB7DEB710927F008FE187BB6E
:1002D0008FEF81BB80EE88BB12BA10927A00109229
:1002E0007B0010927C0010927D0010927E00F7DE61
:1002F00047DF10928F0010928E0010928D001092A6
:100300008600109285001092840010928C0010924A
:100310008B0010928A001092870010928000109239
:100320008100DF91CF9108951F920F920FB60F9227
:1003300011242F933F934F935F936F937F938F93EA
:100340009F93AF93BF93EF93FF93CF93DF93CDB77B
:10035000DEB7809187008F5F809387008091870050
:100360008F3130F110928700809188009091890040
:100370000197909389008093880067DE80918800C0
:10038000909189000097A1F410927F0081E0809302
:100390008000809381008BE0809376008CE08093D6
:1003A00077008DE0809378008EE08093790019BE0D
:1003B00080917F00882309F012BEDF91CF91FF91D9
:1003C000EF91BF91AF919F918F917F916F915F91CD
:1003D0004F913F912F910F900FBE0F901F90189546
:1003E000CF93DF93CDB7DEB780917A008F5F809394
:1003F0007A0080917A00843010F010927A00809117
:100400007A009927F92FE82FE059FF4F90818091CA
:100410007F00892B806E88BB80917E00882319F134
:1004200090917A0080917B009817E9F480917C008C
:100430008F5F80937C0080917C008B3F60F0809187
:100440007D00813019F410927D0003C081E080931B
:100450007D0010927C0080917D00813021F480919C
:100460006A0082BB0FC080917A0099278A589F4FFB
:10047000F92FE82F80819927805A9F4FF92FE82F75
:10048000808182BBDF91CF910895CF93DF93CDB769
:10049000DEB727970FB6F894DEBF0FBECDBF83E05F
:1004A0008B83A4E8B0E0AC83BD83EDE8F0E0EE839D
:1004B000FF83AC81BD81EE81FF818B8101900D9224
:1004C0008A95E1F786B38A838A81898389818072DC
:1004D000882319F010928D0005C080918D008F5FE8
:1004E00080938D0089818074882319F010928E008A
:1004F00005C080918E008F5F80938E008981807807
:10050000882319F010928F0005C080918F008F5FB3
:1005100080938F0080918D00882341F48091840026
:10052000863020F081E080938A0002C010928A0019
:1005300080918E00882341F480918500863020F0E0
:1005400081E080938B0002C010928B0080918F001D
:10055000882341F480918600863020F081E08093EA
:100560008C0002C010928C0027960FB6F894DEBF64
:100570000FBECDBFDF91CF910895CF93DF93CDB75D
:10058000DEB729970FB6F894DEBF0FBECDBF8091BE
:100590007F00882399F080918F00882309F487C019
:1005A00080918D00882309F482C080918E00882379
:1005B00009F47DC085DE19BE64DE79C080918000BB
:1005C000882371F080918F00882349F480918D00F9
:1005D000882329F480918E00882309F401C070DEFD
:1005E00080918C00882371F080E180937F001092CD
:1005F0007E0010928700E4DD82E089BF85E083BF42
:1006000012BE789480918A00882371F080917B00DB
:100610008F5F80937B0081E080937E0080917B00E0
:10062000843010F010927B0080918B00882309F4B5
:100630003EC080917B0099278A589F4FB92FA82FE1
:1006400080917B0099278A589F4FF92FE82F80814E
:100650008F5F8C9381E080937E0080917B0082305D
:1006600099F480917B0099278A589F4FF92FE82FA2
:1006700080818630D8F080917B0099278A589F4FDF
:10068000F92FE82F108212C080917B0099278A5899
:100690009F4FF92FE82F80818A3040F080917B00B6
:1006A00099278A589F4FF92FE82F108218DD299635
:1006B0000FB6F894DEBF0FBECDBFDF91CF91089586
:1006C000CFEDD0E0DEBFCDBFFBDDBFDCDEDE55DF32
:1006D00010927500109274008091740090917500D2
:1006E0008A30910508F0F2CF80918100882331F0A3
:1006F00010927500109274001092810071DEA3DDDB
:10070000809174009091750001969093750080938C
:100710007400E2CFFFCFE199FECF9FBB8EBBE09A82
:1007200099278DB30895E199FECF9FBB8EBBE09AC8
:1007300001960DB29FBB8EBBE09A802D9DB30895AC
:10074000E199FECF9FBB8EBB6DBB0FB6F894E29ACA
:10075000E19A0FBE08954115510571F0A82FB92FE8
:10076000E199FECF7FBB6EBBE09A6F5F7F4F0DB20A
:100770000D9241505040B1F708955527002480FF55
:1007800002C0060E571F660F771F610521F0969570
:1007900087959105A1F7952F802D0895AA1BBB1B66
:1007A00051E107C0AA1FBB1FA617B70710F0A61B71
:1007B000B70B881F991F5A95A9F780959095682FB8
:0807C000792F8A2F9B2F089569
:1007C800407924301912027800107721232B067FF4
:0407D800070B0D0EF0
:00000001FF
